:020000040000FA
:02000000BE2818
:06000A00831603130F3002
:1000100086008113831208000030A000A101703017
:10002000860006080F39A0000E302006031D1B288D
:100030000E30A00094280D302006031D2228003029
:10004000A00094280B302006031D29280F30A000A3
:10005000942807302006031D30280D30A000942876
:10006000B030860006080F39A0000E302006031DB0
:100070003C280730A00094280D302006031D43289B
:100080000830A00094280B302006031D4A280930B0
:10009000A000942807302006031D51280C30A00032
:1000A0009428D030860006080F39A0000E302006B4
:1000B000031D5D280430A00094280D302006031D88
:1000C00064280530A00094280B302006031D6B28FF
:1000D0000630A000942807302006031D72280B303C
:1000E000A0009428E030860006080F39A0000E30EA
:1000F0002006031D7E280130A00094280D30200624
:10010000031D85280230A00094280B302006031D13
:100110008C280330A000942807302006031D932864
:100120000A30A000942808000130A1000800A200B5
:10013000F930A30064006400A30B9A28A20B98284E
:10014000A128640008003730A200B530A300640085
:100150006400A30BA728A20BA5280800A200E83082
:10016000A3006400B328B4286400A30BB128A20B39
:10017000AF28BA28BB28BC286400080007309F00BD
:100180008316031385019F01831205200C20003084
:1001900021060319C62820088500AE20AE20C628F7
:084200003100320033003400EC
:00000001FF
